:10000000E7C001C100C1FFC0FEC0FDC0FCC0FBC015
:10001000FAC0FAC0F8C0F7C0F6C0F5C0F4C0F3C02B
:10002000F2C0F1C0F0C0BAC2C9C2D8C282C681C68D
:1000300003C30EC47EC67DC67CC67BC67AC679C69F
:1000400078C677C63EC3B6C3BBC3A5C2A1C2DBC3D5
:1000500071C501C614C6FFC512C611C610C630C68A
:1000600080C6C9C266C665C664C663C662C661C6C6
:1000700060C65FC65EC65DC65CC65BC65AC659C66C
:1000800072C6BBC2BDC255C6BEC2C5C26CC6B3C273
:10009000C4C24FC6C7C24DC64CC663C6ACC2BFC2FF
:1000A0001B5B306D1B5B324A1B5B303B3066005282
:1000B000656164792E204A75737420636C6F736573
:1000C00020746865207465726D696E616C2E204EB7
:1000D0006F207265736574206E65656465642E0DAE
:1000E0000A005D3A200053656C65637420277374C1
:1000F0006B353030206279207065746B6127206D1C
:100100006F64652E2028313D314D687A20303D46A0
:10011000617374295B002028686578290D0A000D39
:100120000A4F4B2C206D79205357207665727369E6
:100130006F6E206973206E6F773A20005D3A200061
:1001400052657365742074617267657420617420F0
:10015000636F6E6E6563746F7220706F6C6172692D
:100160007479207465737428313D6F6E20303D6F53
:100170006666295B005D3A2000456E746572205307
:10018000572056657273696F6E204D696E6F7220CD
:10019000696E20686578205B005D3A2000456E74CA
:1001A00065722053572056657273696F6E204D61DA
:1001B0006A6F7220696E20686578205B00617672D4
:1001C00075736235303076322D312E32200D0A00B3
:1001D00011241FBECFE5D4E0DEBFCDBF10E0A0E606
:1001E000B0E0ECEEF2E102C005900D92AC36B10742
:1001F000D9F711E0ACE6B0E001C01D92A43AB10716
:10020000E1F7B3D571C8FCCE1F920F920FB60F92D3
:1002100011248F939F9385B391E0892785BB86EE48
:1002200082BF9F918F910F900FBE0F901F901895D6
:10023000A09A91E093BF86EE82BF99BF0895A098DF
:1002400013BE19BE08958BE1A6D785E4A4D70895FF
:10025000DF92EF92FF920F931F93882319F022E011
:10026000E22E02C0EE24E39481E0BAD7182F92E088
:10027000D92E0FEF2DC080EDF82EF10E89E08F15ED
:1002800038F4812F8154863018F080528630E8F49B
:100290000F3F09F400E0812F7ED789E08F1520F011
:1002A0000295007F0F0D10C0812F8154863030F4ED
:1002B000802F8295807F012F075305C0802F829564
:1002C000807F012F0755080FDA9481E089D7182F16
:1002D0001D3039F01A3029F0DD2069F603C081E0C5
:1002E0007FD7EA94EE20D9F7802F1F910F91FF90CE
:1002F000EF90DF9008950F931F93082F80EA90E00E
:1003000058D78DEB91E055D79EDF8DE991E051D71D
:1003100040E150E067E770E08091A10190E0A0D754
:1003200087E790E03CD789E991E043D7802F90DFC1
:100330008F3F11F08093A10186DF89E791E039D7E3
:1003400040E150E067E770E08091A30190E088D73A
:1003500087E790E024D785E791E02BD7802F78DFDF
:100360008F3F11F08093A3016EDF80E491E021D7ED
:10037000FCD54AE050E067E770E090E071D787E78E
:1003800090E00DD78CE391E014D7802F61DF182F18
:100390008F3F31F081E0ECD5112311F480E0E8D5F6
:1003A00052DFE3D5282FE199FECF83E090E09FBB99
:1003B0008EBB2DBB0FB6F894E29AE19A0FBE209146
:1003C000A301E199FECF81E090E09FBB8EBB2DBBE6
:1003D0000FB6F894E29AE19A0FBE2091A101E1993B
:1003E000FECF82E090E09FBB8EBB2DBB0FB6F89492
:1003F000E29AE19A0FBEE199FECF1FBA1EBA84E1DC
:100400008DBB0FB6F894E29AE19A0FBE8FE191E0AE
:10041000D0D640E150E067E770E08091A10190E024
:100420001FD787E790E0BBD68EE2B5D68091A301B7
:10043000803110F480E3AFD640E150E067E770E030
:100440008091A30190E00CD787E790E0A8D686E1E1
:1004500091E0AFD686EE90E0ACD64AE050E067E798
:1004600070E08091A20190E0FBD687E790E097D6FC
:1004700082EE90E09ED6802FEBDE8F3FF1F0882356
:1004800031F41092A201A09813BE19BE08C091E0E9
:100490009093A201A09A93BF86EE82BF99BF20914C
:1004A000A201E199FECF84E090E09FBB8EBB2DBB03
:1004B0000FB6F894E29AE19A0FBEC5DE8FEA90E09B
:1004C00078D61F910F910895CF92DF92EF92FF920D
:1004D0000F931F93DF93CF930F92CDB7DEB7D82E34
:1004E0007B01CB0101978D51914030F080EC8093DE
:1004F000780042E0E42EF12C8BE14DD68D2D4BD6C9
:100500008F2D49D68E2D47D68EE045D695E19D2577
:100510009E259F25A89537E7C32E30E0D32E87016F
:100520000C0D1D1D09C0F6018081998334D6F6019A
:1005300081916F0199819827C016D106A1F7892F63
:100540002AD60F90CF91DF911F910F91FF90EF90DE
:10055000DF90CF9008954F925F926F927F928F922B
:100560009F92AF92BF92CF92DF92EF92FF920F9342
:100570001F93CF93DF93482E8091770090E0FC018A
:100580003197ED31F10508F0D4C3ED5EFF4F0994CA
:10059000DD24D394D0C29924939436C181E0809312
:1005A00077001092780088E08093790060E670E030
:1005B0008AE790E04ED66BE070E0C0C3809178008F
:1005C000883921F480917900F8D478C08F3909F006
:1005D00075C08091790080936C0070C08091780024
:1005E00090E0FC01E058F040E032F10508F0A1C3D2
:1005F000E05DFF4F099481E01AC08091A10114C011
:100600008091A30111C080916D00882369F482E07C
:100610008CD49CD409C089E10AC0F9D405C080916A
:100620006C0002C088E803C08F3F09F482C31092B7
:1006300078008093790020C36091780070917900F0
:10064000272F30E040E050E0A90133272227862FF2
:1006500090E0A0E0B0E0B82FAA2799278827282BA0
:10066000392B4A2B5B2B80917A0090E0A0E0B0E020
:10067000BA2FA92F982F8827282B392B4A2B5B2B91
:1006800080917B0090E0A0E0B0E0282B392B4A2B32
:100690005B2B20936E0030936F004093700050935B
:1006A000710067FF04C081E08093720002C0109265
:1006B00072007093730081E0809374001092780050
:1006C0003BC381E04FD41ED58FE090E047D582E058
:1006D0002CD43CD480936D0031D58091790090E08A
:1006E0003DD580EC8093780080917B00813318F0B9
:1006F00080E380937B0080917C00882319F481E063
:1007000080937C00C0E0D0E04DC0A89580917A0035
:1007100090E024D580917F008ED480917C0090E081
:100720001DD58091800087D480917C0090E016D503
:1007300080918100A1D4182F80917C0090E00ED58B
:100740008091820099D4982F80917E00833031F47B
:1007500080917D00181711F41092780080917E002E
:10076000833031F080917D00981711F41092780059
:1007700080917E00882311F4109278008091780097
:10078000882329F480917B00C82FD0E005C02196F2
:1007900041D484E190E0E2D480917800803C11F46F
:1007A00080E0E0D380917B0090E0C817D90708F47F
:1007B000ACCFC2C280E0D6D3A5D410926D007ECF5C
:1007C000AC9880917A0037D480917B0034D48091AA
:1007D0007C0031D480917D002ED4809179008823D3
:1007E00011F016E906C08091780090E0B7D466CF8A
:1007F000115060E070E080E090EF68D480FF5ECF41
:100800001123B1F75BCF992480917B00843018F4D9
:1008100084E080937B0080917B00813218F080E23D
:1008200080937B0080916E0090916F009093760092
:10083000809375009091780080E020917900A22E3D
:10084000BB24A82AB92A29E1A21621E0B20610F099
:1008500080EC70C280907A00AC9880FE07C001E8FE
:1008600010E0EE24FF24C0E0D0E008C1F1E8EF2E54
:10087000F0E0FF2E16E900E066247724C0E0D0E027
:10088000E2E05E2E7EC0992031F0C0FF04C080916E
:100890007C00886002C080917C00CDD380916E0086
:1008A00090916F000AD4F7018081C5D390917F00A9
:1008B000F7018081981739F060906E0070906F009A
:1008C00080927A0002C050927A00A895992019F47B
:1008D00082E090E043D480917A0082FF21C0909121
:1008E0007F0016E971E0C72ED12CCC22DD2211C089
:1008F000992031F0CC2021F080917E00886002C0E8
:1009000080917E0098D3C301D8D380E0B5D3982FCF
:10091000115080917F009817B1F4112349F713C04B
:1009200083FF0DC016E901C0115060E070E080E067
:1009300090EFCCD380FF07C01123B1F704C08091A2
:100940007B0090E00BD4992011F0C0FF13C0809180
:100950006E0090916F00A0917000B09171000196AF
:10096000A11DB11D80936E0090936F00A093700045
:10097000B0937100112309F400E821960894E11C5A
:10098000F11CCA15DB0508F47ECFD1C0A895809173
:1009900072008823A9F080916E0090916F00892BDE
:1009A00021F080917400882359F08DE465D380E0B4
:1009B00063D38091730060D380E05ED310927400A3
:1009C000992031F0C0FF04C080917C00886002C093
:1009D00080917C0030D380916E0090916F006DD338
:1009E000F801808128D390917F00F80180819817C9
:1009F00029F0E0906E00F0906F0006C080917A00C0
:100A00008078806180937A00992011F1C0FF33C013
:100A100080916E0090916F00A0917000B091710074
:100A20000196A11DB11D80936E0090936F00A0935D
:100A30007000B0937100A070B0708F5F9F4FA040A6
:100A4000B040C9F4809173008F5F8093730013C02E
:100A500080916E0090916F00A0917000B091710034
:100A60000196A11DB11D80936E0090936F00A0931D
:100A70007000B093710021960F5F1F4FCA15DB0500
:100A800008F484CF80917A0087FF4CC080917D006C
:100A9000D2D280917500909176000FD380E0CBD2B6
:100AA000992019F481E090E059D380917A0085FF74
:100AB00023C0E114F10401F190917F0016E9E701F0
:100AC000C170D0700FC0209721F080917E008860A7
:100AD00002C080917E00AFD2C701EFD280E0CCD2BD
:100AE000982F115080917F00981719F4112359F70E
:100AF0001BC01123C9F016C086FF10C016E901C043
:100B0000115060E070E080E090EFE0D280FF03C021
:100B10001123B1F70BC0112349F004C080917B0071
:100B200090E01CD300E003C000E801C001E800939E
:100B3000780002C1DD249091780080E02091790056
:100B4000C22FD0E0C0907A00C82BD92B21E0C93148
:100B5000D20710F0C8E1D1E0AC9869E7E62E60E07A
:100B6000F62E00E010E058E0B52EBC2867C0A8952E
:100B7000809172008823A9F080916E0090916F009F
:100B8000892B21F080917400882359F08DE474D270
:100B900080E072D2809173006FD280E06DD21092AB
:100BA0007400DD2021F000FF02C08B2D01C08C2DD0
:100BB00042D280916E0090916F007FD280E05CD233
:100BC000F7018083DD2011F100FF33C080916E00BA
:100BD00090916F00A0917000B09171000196A11DDD
:100BE000B11D80936E0090936F00A0937000B0933E
:100BF0007100A070B0708F5F9F4FA040B040C9F4EB
:100C0000809173008F5F8093730013C080916E009A
:100C100090916F00A0917000B09171000196A11D9C
:100C2000B11D80936E0090936F00A0937000B093FD
:100C300071000F5F1F4F0894E11CF11C0C171D077A
:100C400008F495CFBE016D5F7F4F10927800C958B0
:100C5000DF4F1A8273C0AC9880917800ECD18091FC
:100C60007900E9D180917A00E6D180917B00E3D1CF
:100C7000109278001092790063E070E05FC0AC9849
:100C800009E710E0C1E0D0E0F8018081F5D1282F1C
:100C90008091780090E08C179D0711F420937900E3
:100CA00085E090E05BD20F5F1F4F2196C530D105E4
:100CB00059F71092780010927A0064E070E03EC01C
:100CC000F0907900E0907A00AC9810E000E01BC052
:100CD00085E090E043D20E1578F01F1568F4E02F00
:100CE000F0E0E958FF4F8481C7D1E12FF0E0E958E7
:100CF000FF4F82831F5F06C0E02FF0E0E958FF4FEF
:100D0000848199D10F5F80917800081708F304C09F
:100D1000E958FF4F12821F5FE12FF0E01F15C0F36B
:100D2000BF016D5F7F4F10927800E958FF4F12822C
:100D300005C089EC8093780062E070E0842DC4DB0C
:100D4000DF91CF911F910F91FF90EF90DF90CF90A7
:100D5000BF90AF909F908F907F906F905F904F90DB
:100D6000089580E064CC82E062CCAF92BF92CF92D3
:100D7000DF92EF92FF920F931F93CF93DF93BA9A74
:100D800010E01F5FC29A84E190E0E8D1C2988DE73D
:100D900090E0E4D11630A9F7F6D1C2987894E8D162
:100DA0008AE08093A30182E08093A101E199FECFC4
:100DB0001FBA1EBAE09A8DB3843141F5E199FECF96
:100DC00081E090E09FBB8EBBE09A8DB38093A3013E
:100DD000E199FECF82E090E09FBB8EBBE09A8DB39D
:100DE0008093A101E199FECF84E090E09FBB8EBB90
:100DF000E09A8DB38093A201E199FECF83E090E069
:100E00009FBB8EBBE09A8DB3B3D002C01092A201FB
:100E10008091A201882321F4A09813BE19BE06C0B8
:100E2000A09A91E093BF86EE82BF99BFCC24AA24FA
:100E300003C0C12E06C0CC24BB24EE24FF24C0E096
:100E4000D0E081E0CDD1182F8B3149F401E09BE156
:100E5000D92E80E0C5D1182F0130F9F41AC08D3099
:100E600011F08A3041F72196AA2039F41A3051F452
:100E70008DE0C81639F4AA24A394C430D105C9F66C
:100E800081E004C0C230D105A1F680E034DAC12E81
:100E9000D6CFD826B82E02E0DCCF023029F4D826EF
:100EA000F82EEE2403E0D5CF033031F4D82690E0BD
:100EB000E82AF92A04E0CDCF043041F4D8268E3058
:100EC00009F0BFCF05E0C0E0D0E0C3CF0530B9F4F2
:100ED000CE15DF0508F0AFCF81E0C831D80708F0A4
:100EE000AACFD126FE01E958FF4F10832196A8957D
:100EF000CE15DF0509F0ADCF7E0106E0AACF0630A2
:100F000009F099CF8D1531F4EF2821F0A8958B2D9C
:100F100022DB91CF80EB8093770081EC8093780087
:100F200062E070E08B2DD0DA86CF8F70806C87B94D
:100F300087E886B9369A3699FECF24B145B1942F09
:100F400080E030E0282B392BC9010895880F991FC4
:100F5000880F991F60E370E0B3D1862F08958091C8
:100F60009E01089580939E010895809169000895DF
:100F70008093690008951F93809169008823C9F0C8
:100F8000A398AB988CE090E0E9D082E0CEDFDEDF82
:100F9000182FA39AAB988CE090E0E0D082E0C5DFF8
:100FA000D5DF682FA398AB9820E0812F7DD18430C6
:100FB00008F021E0822F1F9108958A3028F08FE0F9
:100FC00080936B008AEF1EC0873028F087E0809303
:100FD0006B0088E717C0833028F083E080936B00B4
:100FE00080E510C0823021F480936B0082E30AC058
:100FF000882329F081E080936B0086E003C0109283
:101000006B0081E080936A0080916B00089580916D
:101010006B000895AC9880916A00982F9A95F1F72B
:10102000982F9A95F1F7AC9A982F9A95F1F78A959F
:10103000F1F7AC980895582F40916A0090E828E0A5
:1010400030E071E063E0892F852311F0A99A01C097
:10105000A998842F8A95F1F7872F8A95F1F7AC9A92
:10106000842F8A95F1F7862F8A95F1F79695AC989B
:101070002150304041F70895682F50916A0090E860
:1010800040E028E030E073E0892F862311F0A99A30
:1010900001C0A998852F8A95F1F79D99492BAC9AA3
:1010A000852F8A95F1F7872F8A95F1F79695AC9859
:1010B0002150304049F7842F08951F93182FAC9882
:1010C000892FB9DF812FB7DF1F910895EF92FF922B
:1010D0000F931F937B018C01AC98892F9927AA2726
:1010E000BB27A9DFC801AA27BB27A5DFBB27A12FE4
:1010F000902F8F2DA0DF8E2DBFDF1F910F91FF90BE
:10110000EF900895A49AAC98AB9AA598AD98A4983E
:10111000AC98A198A99884E190E020D0A398AB98CE
:101120000895AB9A80916A00982F9A95F1F78A9565
:10113000F1F7AB9884E190E011D00895A39AAB9AAF
:10114000A598A19AA998A49AAC988AE090E006D0B4
:10115000AB9884E190E002D0E4DF089522ED3DE019
:1011600004C0F9013197F1F701970097D1F708957D
:101170002FE088E190E00FB6F894A89581BD0FBEEE
:1011800021BDA895089510BC87E089B988E18AB986
:1011900086E880BD08955D9BFECF8CB90895FC0163
:1011A00004C05D9BFECF8CB9319680818823C9F73E
:1011B000089503C05D9BFECF2CB9FC0101962491DC
:1011C0002223C1F7089503C0882309F0A8955F9BE7
:1011D000FBCF8CB1089501C08CB15F99FDCF08950C
:1011E000EF92FF920F931F93F82E01E0EE24E39409
:1011F00028C0FF2009F0A895B2DE882341F0809135
:101200009F018111C29A1092A00101E01AC000232F
:10121000B9F41091A00182E088DE98DE810F8695F6
:101220008093A0018A3020F4C29810929F0108C0D8
:10123000C29906C0A0DE882319F0C29AE0929F01ED
:101240000F5F5F9BD6CF8CB11F910F91FF90EF90F6
:101250000895FB01DC0101900D920020E1F7089553
:10126000FB019F0142306CF045325CF4642F77271C
:1012700027D0805D8A330CF0895D8193CB01009784
:10128000A9F71082C90100C0DC01FC01672F719130
:101290007723E1F7329704C07C916D93708362915C
:1012A000AE17BF07C8F30895991B79E004C0991FD2
:1012B000961708F0961B881F7A95C9F780950895B0
:1012C000AA1BBB1B51E107C0AA1FBB1FA617B7076C
:1012D00010F0A61BB70B881F991F5A95A9F7809588
:0C12E0009095BC01CD010895F894FFCF5B
:0C12EC004156524953505F320001060188
:00000001FF
